:0600000000308A000F2809
:10000800FF00030883120313BC000A08BD007E0822
:10001800BE008A11F92EF901FA01FB01FC01FD016C
:040028008A11C02C4D
:10020000FE00FE1F082983137E18831700080800CC
:100210008A00040882000034383467342C343834BF
:10022000653436342C343834643436342C34383431
:10023000633436342C34323467342C3438346734F5
:100240002C343834653436342C3438346434363411
:100250002C343834633436342C34323461342C3416
:10026000383461342C343834663436342C343834F1
:10027000653436342C343834643436342C343834E1
:1002800062342C34383467342C34383462342C34AF
:100290003834643436342C34383467342E343634BD
:1002A0002C3431343634673436342C3438346634B4
:1002B00036342C343834643436342C3432346534A7
:1002C00036342C34383467342C343834653436348E
:1002D0002C343834643436342C3438346334363483
:1002E0002C34323467342C3431343634663423348D
:1002F0002C34383467342C343834653436342C3468
:100300003834643436342C343834633436342C3452
:10031000323461342C34383461342C34383466341B
:1003200036342C343834653436342C343834643430
:1003300036342C343834673436342C343134363453
:10034000673436342C34313436346634233436341E
:100350002C3431343634673436342C34313436343A
:100360006634233436342C343134363467343634FE
:100370002C34313436346734233436342C34383426
:1003800061342E3436342C343134363467343634D8
:100390002C343834653436342C34383464343634C0
:1003A0002C34633436342C34673436342C343834BB
:1003B000653436342C343834653436342C3438349F
:1003C00065342E3436342C343134363464342334AA
:1003D00036342C343834653436342C34383465347F
:1003E00036342C34383465342E3436342C343134AD
:1003F00036346434233436342C343834653436346B
:100400002C343834673436342C34383463342E3456
:1004100036342C3431343634643436342C3432347B
:10042000653436342C343834663436342C3438342D
:10043000663436342C34383466342E3436342C3426
:1004400031343634663436342C3438346634363409
:100450002C343834653436342C34383465343634FE
:100460002C3431343634653436342C34313436342B
:10047000653436342C343834653436342C343834DE
:10048000643436342C343834643436342C343834D0
:10049000653436342C343234643436342C343234CB
:1004A00070342C34383461342E342C343834633482
:1004B0002E3436342C343134363464342E343634DD
:1004C0002C3431343634643436342C343834633498
:1004D0002E3436342C343834673423342C343134CD
:1004E0003634673423342C34313436346334363480
:1004F0002C343134363470342C3464342E34363465
:100500002C34383470342C343834633436342C344E
:100510003134363461342C34383462342C34313450
:10052000363461342C34383467342E342C3432343D
:1005300063342E3436342C34383470342C3438341C
:10054000633436342C3431343634633436342C341A
:10055000383463342E3436342C34313436347034F9
:100560002C34383462342C343134363462342C3404
:10057000383462342E342C34383461342C343134F1
:10058000363462342C34383461342C3465342E34AF
:100590002C34383470342C34383461342C343134C5
:1005A000363462342C34383461342C343834653485
:1005B0002E342C34383467342C343134363470349F
:1005C0002C34383461342C343134363462342C34A5
:1005D000383461342C3466342E342C34383470344E
:1005E0002C34383464342C34383465342E342C3480
:1005F0003134363466342C343134363467342C3468
:10060000383470342C34383461342C34313436344A
:1006100067342C34383464342C3431343634653413
:100620002C343134363466342C343134363470342E
:100630002C34323467342C34323470342C3431342A
:100640003634643436342C34653436342C3438340F
:1006500070342C34653436342C34383464343634C5
:100660002C34383470342C34383461342C343834ED
:10067000653436342C343834653436342C343834DC
:100680006634233436342C3464342E3436342C34EB
:10069000383462342C34383462342C343834653491
:1006A00036342C343834653436342C3466342334C0
:1006B00036342C3464342E3436342C3438346234AA
:1006C0002C3438346334233436342C3438346434A2
:1006D00036342C3438346334233436342C343234C6
:1006E00062342E342C3431343634653436342C3480
:1006F0006634233436342C34383470342C34653436
:100700002E3436342C34383470342C34383462344B
:100710002C3438346634233436342C34383467344B
:1007200036342C3438346634233436342C34323472
:10073000653436342C343834643436342C3438341C
:100740006334233436342C343834643436342C3423
:1007500038346334233436342C346334233436341D
:100760002C343834643436342C34383470342C34EB
:1007700038346334233436342C34383470342C34E5
:10078000323461342C3431343634643436342C34DD
:10079000653436342C34383470342C346534363483
:1007A0002C343834643436342C34383470342C34AB
:1007B000383461342C343834653436342C3438349D
:1007C000653436342C3438346634233436342C349F
:1007D00064342E3436342C34383462342C34383487
:1007E00062342C343834653436342C34383465343F
:1007F00036342C346634233436342C3464342E347A
:1008000036342C34383462342C3438346334233462
:1008100036342C343834643436342C34383463343D
:10082000233436342C34323462342E342C34313484
:100830003634653436342C346634233436342C3430
:10084000383470342C3465342E3436342C34383407
:1008500070342C34383462342C34383466342334D5
:1008600036342C343834673436342C3438346634E7
:10087000233436342C343234653436342C34383422
:10088000643436342C3438346334233436342C34E2
:100890003834643436342C343834633423343634C6
:1008A0002C346334233436342C34383464343634C2
:1008B0002C34383470342C343834633423343634A4
:1008C0002C34383470342C3461342C343234703459
:1008D0002C3464342C3467342C34383467342C345E
:1008E000383461342C34383467342C34383466343A
:1008F00023342C3465342C3465342C3465342C3456
:1009000061342C34383461342C34383462342C342F
:10091000383461342C34383467342C34663423341E
:100920002C3464342C3464342C3462342C34383415
:1009300062342C343834633436342C3438346234F2
:100940002C34383461342C3467342C3465342C34F2
:1009500064342C3465342C3461342C3466342334C0
:100960002C34323467340034D7308316810083123C
:100970000B118B169001900A0C1083160C140800B2
:10098000AA01AB01A401A501A601A701A801A90123
:10099000A201A301A001A1010530A200A30104301E
:1009A000A000A1016430F000831605118312031723
:1009B0009E010313F901B42483120B178B1723082C
:1009C000A5002208A4000C302A0784000130031877
:1009D00002302B078A1100218A11333A031DFF2CA4
:1009E0000D302A0784000130031802302B078A11CA
:1009F00000218A11323A031DFF2C20301A2D0C30B1
:100A00002A0784000130031802302B078A110021C5
:100A10008A11313A031D212D0D302A07840001303F
:100A2000031802302B078A1100218A11363A031D60
:100A3000212D1030A600A7010230AA070318AB0A27
:100A4000672D0C302A0784000130031802302B0771
:100A50008A1100218A11383A031D302D08304D2D9E
:100A60000C302A0784000130031802302B078A114A
:100A700000218A11343A031D3F2D04304D2D0C30D6
:100A80002A0784000130031802302B078A11002145
:100A90008A11323A031D4F2D0230A6005E2D0C3014
:100AA0002A0784000130031802302B078A11002125
:100AB0008A11313A031D632DA601A60AA701AA0ACD
:100AC0000319AB0A672D2108A7002008A6000D30E6
:100AD0002A0784000130031802302B078A110021F5
:100AE0008A11233A03198A2DC82DE630A80029302F
:100AF000882D3B30A8002330882D6330A8001F309C
:100B0000882D6530A8001A30882D8830A80017304D
:100B1000A900A32D0C302A078400013003180230ED
:100B20002B078A1100218A11613A0319752D023AA7
:100B30000319792D073A03197D2D023A0319812DE6
:100B4000013A0319852D0230AA070318AB0AED2DCF
:100B50006430A8002C30C32D8B30A8002730C32D63
:100B60005330A8002530C32D4130A8002130C32DBB
:100B7000A030A8001D30C32DF630A8001B30C32DB7
:100B8000EA30A8001830A900EA2DA801A901EA2D31
:100B90000C302A0784000130031802302B078A1119
:100BA00000218A11613A0319A82D033A0319AC2DCB
:100BB000013A0319B02D073A0319B42D013A03196C
:100BC000B82D033A0319BC2D013A0319C02D173A69
:100BD0000319C52DAA0A0319AB0A0C302A07840091
:100BE0000130031802302B078A1100218A112E3A96
:100BF000031D012E8030A6070318A70AAA0A0319AD
:100C0000AB0A0C302A0784000130031802302B078E
:100C10008A1100218A11343A031D102E04303C2E13
:100C20000C302A0784000130031802302B078A1188
:100C300000218A11353A031D1F2E05303C2E0C3041
:100C40002A0784000130031802302B078A11002183
:100C50008A11363A031D2E2E06303C2E0C302A0700
:100C600084000130031802302B078A1100218A11F9
:100C7000373A031D412E0730A400A501AA0A031923
:100C8000AB0A0C302A0784000130031802302B070E
:100C90008A1100218A112E3A031D552E8030A60795
:100CA0000318A70AAA0A0319AB0A2708B2002608E4
:100CB000B10024088313B0002908AF002808AE0053
:100CC0008A11A5262B08AD002A08AC00AA0A031930
:100CD000AB0A0C3E84000130031802302D078A1144
:100CE00000218A112C3A0319DF2C7B087A04031D9A
:100CF000752EF9017A2EBA01BB01380837040319A1
:100D0000A02EB901B90A0310B81B8A2EB70DB80D71
:100D1000822E0310BA0DBB0D38083602031D922E29
:100D200037083502031C9C2E3708B5023808031C0F
:100D3000B603B6023A140310B80CB70CB90B892EDF
:100D40003B08B6003A08B5000800B72E0310AF0CF8
:100D5000AE0C0310AF0CAE0CC42EAE0EAF0E0F30A7
:100D6000AE052F08F039AE040F30AF05C42E3008A1
:100D7000043A0319C42E013A0319A92E033A0319A0
:100D8000A62E013A0319AD2E7B087A04031DC42E4A
:100D9000F9012F082E040319D72EFF30AE06AF0637
:100DA0002E08FC00B301FF302F05B400FD007F309A
:100DB0003105B700B801FF30B500B6017B26360813
:100DC000FB003508FA00B11FF22E7B08B4007A0848
:100DD000B3000310B40CB30C3308FA070318FB0A72
:100DE0003408FB072F082E0403190800F901F90A3B
:100DF00008000B1D062F700881007B087A04031978
:100E0000052F0130FA02031CFB030B110C1C142FDD
:100E1000F90803190E2F043085060F2F05117D08E0
:100E20008F007C088E000C103E08FE003D088A00F2
:0A0E30003C088300FF0E7F0E09004E
:00000001FF
